:10000000008000106D010000E1010000E701000028
:10001000ED010000F3010000F90100000000000004
:10002000000000000000000000000000FF010000D0
:1000300005020000000000000B0200004D0300005C
:100040001102000011020000110200001102000064
:100050001102000011020000110200001102000054
:100060001102000011020000110200001102000044
:100070001102000011020000110200001102000034
:100080001102000011020000110200001102000024
:100090001102000011020000110200001102000014
:1000A0001102000011020000110200001102000004
:1000B00011020000110200001102000011020000F4
:1000C0001102000011020000110200006C0B000080
:1000D00000000010040000006C0B000000C00720AE
:1000E00000000000040000103400000000C00720E1
:1000F0000000000080B489B000AFF860B9607A6099
:10010000BB68FB61FB68BB6100237B610AE0BA69E5
:10011000131DBB61FB69191DF96112681A607B69C7
:1001200004337B617A697B689A42F0D300BF24373D
:10013000BD4680BC704780B485B000AF7860396040
:100140007B68FB600023BB6007E0FB681A1DFA6058
:1001500000221A60BB680433BB60BA683B689A42ED
:10016000F3D300BF1437BD4680BC704780B584B060
:1001700000AF184BFB6013E0FB681A1DFA601B68A8
:10018000BB60FB681A1DFA601B687B60FB681A1D68
:10019000FA601B683B603A687968B868FFF7AAFFA5
:1001A000FB680D4A9342E7D30DE0FB681A1DFA6025
:1001B0001B687B60FB681A1DFA601B683B6039682E
:1001C0007868FFF7B8FFFB68044A9342EDD300F06C
:1001D000C7FCFEE7CC000000E4000000F4000000D3
:1001E00080B400AFFEE780B400AFFEE780B400AF9C
:1001F000FEE780B400AFFEE780B400AFFEE780B456
:1002000000AFFEE780B400AFFEE780B400AFFEE7CA
:1002100080B400AFFEE700BFFFFFFFFFFFFFFFFF5F
:10022000FFFFFFFFFFFFFFFFFFFFFFFFFFFFFFFFDE
:10023000FFFFFFFFFFFFFFFFFFFFFFFFFFFFFFFFCE
:10024000FFFFFFFFFFFFFFFFFFFFFFFFFFFFFFFFBE
:10025000FFFFFFFFFFFFFFFFFFFFFFFFFFFFFFFFAE
:10026000FFFFFFFFFFFFFFFFFFFFFFFFFFFFFFFF9E
:10027000FFFFFFFFFFFFFFFFFFFFFFFFFFFFFFFF8E
:10028000FFFFFFFFFFFFFFFFFFFFFFFFFFFFFFFF7E
:10029000FFFFFFFFFFFFFFFFFFFFFFFFFFFFFFFF6E
:1002A000FFFFFFFFFFFFFFFFFFFFFFFFFFFFFFFF5E
:1002B000FFFFFFFFFFFFFFFFFFFFFFFFFFFFFFFF4E
:1002C000FFFFFFFFFFFFFFFFFFFFFFFFFFFFFFFF3E
:1002D000FFFFFFFFFFFFFFFFFFFFFFFFFFFFFFFF2E
:1002E000FFFFFFFFFFFFFFFFFFFFFFFFFFFFFFFF1E
:1002F000FFFFFFFFFFFFFFFFFFFFFFFFFFFFFFFF0E
:1003000080B400AF0F4BDB680F4AA2FB0323DB086E
:100310000C4A013B53600B4B00229A60094A136858
:1003200043F004031360074A136843F001031360AA
:10033000044A136843F00203136000BFBD4680BC4B
:10034000704700BF10E000E0CDCCCCCC80B400AF53
:10035000044B1B68013B034A136000BFBD4680BCD1
:10036000704700BF0000001080B400AF3C4B20225B
:100370001A6000BF3A4B1B6803F04003002BF9D012
:10038000384B03221A60384B00221A60374B002288
:100390001A60374B01221A60364B374A1A60374BC6
:1003A000AA221A60354B55221A60354B01221A6079
:1003B000324BAA221A60314B55221A6000BF314BD2
:1003C0001B6803F08063002BF9D02D4B03221A60C9
:1003D0002A4BAA221A60294B55221A6000BF294BCA
:1003E0001B6803F04073002BF9D0274B23221A60BF
:1003F000264BAA221A60254B55221A60244B012253
:100400001A60224BAA221A60204B55221A6000BFA4
:10041000204B1B6803F48063002BF9D01C4B032294
:100420001A601A4BAA221A60184B55221A6000BF94
:10043000184B1B6803F44073002BF9D0164B174A76
:100440001A60174B00221A60164B1B6823F4704386
:10045000144A43F48043136000BFBD4680BC70471C
:10046000A0C10F4004C10F40A8C10F40ACC10F4054
:100470000CC10F4084C00F40630005008CC00F40CA
:1004800080C00F4088C00F40A4C00F40ACC00F40D8
:10049000A0C00F40A8C00F40C4C00F40DE87280492
:1004A000C8C10F4000C00F4080B584B000AFF860F5
:1004B000B9607A603B603B6A00229A623B6A002224
:1004C0001A633B6ABA691A624EF66022BB6992FBF4
:1004D000F3F2FB6992FBF3F31A463B6A5A6241223C
:1004E000396AF86800F046F90346B3F1FF3F02D1DC
:1004F0004FF0FF3327E04222396AB86800F03AF93A
:100500000346B3F1FF3F02D14FF0FF331BE043221C
:10051000396A786800F02EF90346B3F1FF3F02D143
:100520004FF0FF330FE04422396A386800F022F9B7
:100530000346B3F1FF3F02D14FF0FF3303E0386AC7
:1005400000F076F9002318461037BD4680BDFFFF46
:1005500080B584B000AF78603960786800F002FB45
:10056000F8607B68002B02DB3B680122DA627B6863
:10057000002B3ADA3B680022DA6236E01E4B1B6839
:10058000002B32D11C4B06221A603B68DB6A012B20
:100590000ED13B689B6A5A1C3B689A623B689A6A18
:1005A0003B681B6A9A4210D13B6800229A620CE0B9
:1005B0003B689B6A002B03D13B681A6A3B689A62CE
:1005C0003B689B6A5A1E3B689A62FB68013BFB6072
:1005D0003B689B6A5A4203F0030302F0030258BFD0
:1005E00053423968184600F009F8FB68002BC5DC57
:1005F00000BF1037BD4680BD0000001080B582B03E
:1006000000AF786039607B68032B00F2AF8001A2F5
:1006100052F823F02506000077060000C906000006
:100620001B0700003B681B68D8B23B685B68DBB205
:100630000122194600F02EFA3B689B68D8B23B684D
:10064000DB68DBB20022194600F024FA3B681B6924
:10065000D8B23B685B69DBB20122194600F01AFA96
:100660003B689B69D8B23B68DB69DBB20022194664
:1006700000F010FA7AE03B681B68D8B23B685B6810
:10068000DBB20022194600F005FA3B689B68D8B23D
:100690003B68DB68DBB20122194600F0FBF93B68DE
:1006A0001B69D8B23B685B69DBB20122194600F0D6
:1006B000F1F93B689B69D8B23B68DB69DBB2002289
:1006C000194600F0E7F951E03B681B68D8B23B6877
:1006D0005B68DBB20022194600F0DCF93B689B68DE
:1006E000D8B23B68DB68DBB20122194600F0D2F9D0
:1006F0003B681B69D8B23B685B69DBB200221946D4
:1007000000F0C8F93B689B69D8B23B68DB69DBB293
:100710000122194600F0BEF928E03B681B68D8B2F8
:100720003B685B68DBB20122194600F0B3F93B6815
:100730009B68D8B23B68DB68DBB20022194600F048
:10074000A9F93B681B69D8B23B685B69DBB2002240
:10075000194600F09FF93B689B69D8B23B68DB699A
:10076000DBB20122194600F095F900BF00BF08373F
:10077000BD4680BD80B487B000AFF860B960134655
:10078000FB71FB680D3B032B1ED801A252F823F02E
:10079000BF070000B5070000AB070000A10700007D
:1007A00002233B6108237B6111E001233B6112239B
:1007B0007B610CE001233B6115237B6107E0012392
:1007C0003B6118237B6102E04FF0FF332BE0FB79A4
:1007D000413B032B26D801A252F823F0ED0700007D
:1007E000FB07000009080000170800003A69BB6811
:1007F0001A607A69BB685A6014E03A69BB689A600B
:100800007A69BB68DA600DE03A69BB681A617A6997
:10081000BB685A6106E03A69BB689A617A69BB684D
:10082000DA6100BF002318461C37BD4680BC704704
:1008300080B582B000AF78607B681B68D8B27B68F7
:100840005B68DBB20022194600F072F87B681B6817
:10085000D8B27B685B68DBB20122194600F0E0F891
:100860007B681B68D8B27B685B68DBB200221946E4
:1008700000F0A4F87B689B68D8B27B68DB68DBB2C9
:100880000022194600F054F87B689B68D8B27B6858
:10089000DB68DBB20122194600F0C2F87B689B6876
:1008A000D8B27B68DB68DBB20022194600F086F81C
:1008B0007B681B69D8B27B685B69DBB20022194692
:1008C00000F036F87B681B68D8B27B685B68DBB2E7
:1008D0000122194600F0A4F87B681B69D8B27B6836
:1008E0005B69DBB20022194600F068F87B689B69FF
:1008F000D8B27B68DB69DBB20022194600F018F839
:100900007B689B69D8B27B68DB69DBB20122194640
:1009100000F086F87B689B69D8B27B68DB69DBB244
:100920000022194600F04AF800BF0837BD4680BDD6
:1009300080B483B000AF0346FB710B46BB71134616
:100940007B71FB795B00DAB2BB791B09DBB2134424
:10095000FB71BB7903F00F03DBB25B00BB71FB796A
:100960009B0003F1804303F530331A68BB79032100
:1009700001FA03F3DB431946FB799B0003F1804343
:1009800003F530330A401A60FB799B0003F1804382
:1009900003F530331A687979BB7901FA03F3194604
:1009A000FB799B0003F1804303F530330A431A605F
:1009B00000BF0C37BD4680BC7047FFFF80B483B0DA
:1009C00000AF0346FB710B46BB7113467B71FB798D
:1009D0009A00124B13441A68BB79012101FA03F300
:1009E000DB431846FB7999000C4B0B4402401A601C
:1009F000FB799A00094B13441A687979BB7901FA9B
:100A000003F31846FB799900044B0B4402431A6028
:100A100000BF0C37BD4680BC704700BF68C00240B5
:100A200080B483B000AF0346FB710B46BB71134625
:100A30007B71FB79DB00FB71FB799B0003F10053B9
:100A400003F51C231A68BB79012101FA03F3DB4388
:100A50001946FB799B0003F1005303F51C230A4060
:100A60001A60FB799B0003F1005303F51C231A68FD
:100A70007979BB7901FA03F31946FB799B0003F1FD
:100A8000005303F51C230A431A6000BF0C37BD4610
:100A900080BC704780B483B000AF0346FB710B4647
:100AA000BB7113467B71FB79DB00DBB20533FB7155
:100AB000FB799B0003F1005303F51C231A68BB79F3
:100AC000012101FA03F3DB431946FB799B0003F193
:100AD000005303F51C230A401A60FB799B0003F1C5
:100AE000005303F51C231A687979BB7901FA03F3E3
:100AF0001946FB799B0003F1005303F51C230A43BD
:100B00001A6000BF0C37BD4680BC704780B584B00A
:100B100004AFFFF729FCFFF7F3FB104B02933C23D4
:100B20000193C823009310230F220E210D20FFF7FD
:100B3000BBFC002201210220FFF7FAFE0122012165
:100B40000220FFF76DFF002201210220FFF736FF90
:100B50000249B420FFF7FCFCFAE700BF04000010D4
:0C0B6000FFF7D4BF0028B8BF4042704728
:040B6C00060000007F
:040000030000016D8B
:00000001FF
